:020000040000FA
:10000000262A10302D2121302D2102302D21803043
:100010002D2100302D2108302D2100302D2156308A
:100020002D21080010302D2100302D2103302D21ED
:1000300080302D2100302D2108302D2100302D2140
:100040001A302D2108004B30BC204930BC204E30E6
:10005000BC205430BC204930BC203A30BC20203079
:10006000BC202030BC2008004230BC204530BC20E1
:100070004E30BC205430BC204930BC203A30BC202B
:100080002030BC202030BC2008003A08C1003808CD
:10009000C000E7212030BC203B08C1003908C00067
:1000A000E72108003E08C1003C08C000E7212030DD
:1000B000BC203F08C1003D08C000E72108008400C3
:1000C0000008A500840A0008A600840A0008A7000A
:1000D000840A0008A8000800840025088000840A1B
:1000E00026088000840A27088000840A28088000E7
:1000F00008005630BC206930BC206330BC2073300F
:10010000BC207930BC207330BC202030BC20203093
:10011000BC205630BC202030BC203130BC202E30DA
:10012000BC203030BC202E30BC203030BC20080039
:100130000130C52008000230C5200800033904380A
:10014000C520080007390838C52008003F39403865
:10015000C52008008038C52008008316FF308600BF
:100160008312051085140515060805117F398510C1
:1001700083168601831208009000E720851005147D
:10018000051510088600051108009000E72085106D
:100190000510051510088600051108004108031D0B
:1001A000D4282B30960008002D30960008009000CF
:1001B000100E0F39F63E0318073E3A3E9400100821
:1001C0000F39F63E0318073E3A3E930008008316A7
:1001D000FF308600831205108514051506080511E9
:1001E0008039031DE72885108316860183120800D5
:1001F000A5309100910BFA2808009200F820920B8C
:10020000FE28080085011E30FD203830C520003052
:10021000A22098200430A22002309E200800000076
:100220000000A20B0F2908000830A0000512831659
:10023000051283120130A2000F21831605168312C6
:100240000000000005081039FF3EA10C0B30A20091
:100250000F21A00B162921080800A1000830A000DA
:1002600005128316051283120130A2000F21A10C82
:10027000031805160D30A2000F21831605168312F0
:100280000000A00B30290800051283160512831206
:100290007730A2000F218316051683120C30A200BE
:1002A0000F210000000005081039A3003B30A20018
:1002B0000F2123080800410803190800C003C009E2
:1002C00008004421031D8E296D2955302D21012060
:1002D000742955302D211220742917186529971873
:1002E0006929CC302D217429BE302D210930A3007D
:1002F0004030840014218000840AA30B7A29442111
:10030000CC302D2144302D211421031D8429410896
:1003100003198D29013E031D8E2900340134442127
:1003200033302D210830A3003030840014218000A8
:10033000840AA30B96290800FF30B800B900BB005F
:10034000BC00BD00BF00BA01BE0108002808031DA3
:10035000B1294108031D080026084002031C0800BB
:10036000B82941080319B8292608400203180800D3
:100370004008A6004108A80008002708031DC82956
:100380004108031DCF2925084002031CCF2908007E
:1003900041080319080025084002031C0800400812
:1003A000A5004108A70008004330BC20DF30BC2076
:1003B00008000830A300303084000008D72014085B
:1003C000BC201308BC20840AA30BDD290800CE2022
:1003D0001608BC204008CD003530950001304D0591
:1003E000031DF429303095000310CD0CCC010422FC
:1003F00030304A07BC2030304B07BC202E30BC20A8
:100400001508BC20D42108004C08F13E4C07C90057
:1004100049074907FD3ECA004D0E0F39CA07CA07F2
:100420004C07FB3CCB00CB07CB07CB074D080F3964
:10043000CB070A30CB07CA03031C1A2ACA07C90311
:10044000031C1E2AC907031C222A080083018B01F2
:100450008A01850186018316F83085000030860008
:100460008117831281150114811401159C2101301B
:1004700098000221982061210030AA207920403084
:10048000AA208F21D92164006300640063009820B2
:10049000011081100130970061215B2138305F200D
:1004A000A621BD2138306C200030AA20181C5B2A00
:1004B0002320E7215E2A981C5E2A452002309700FF
:1004C00061215B213C305F20A621BD213C306C20A6
:1004D0004030AA20181C6F2A3420E721722A981C69
:1004E000722A5220640063000310980D181D4A2AD6
:0604F000013098004A2AC9
:02400E00FD3F74
:00000001FF
